:0400000002006E325A
:03000B00020136B9
:0100130032BA
:01001B0032B2
:0300230002018057
:01002B0032A2
:01003300329A
:03003B00021FDFC2
:01004300328A
:01004B003282
:01005300327A
:01005B003272
:01006300326A
:03006B000202B5D9
:0300C7000200CA6A
:0500CA001200CF80FED2
:0E00CF0043A2807584007585007591AE759210
:0E00DD005D75A40075A53475B10075B201758E
:0E00EB0080FF75900D75A0FE75B00353A7FE43
:0D00F90012218B900170E0FABAFF02800224
:020106008A96D7
:0701080012016C121FEE1240
:08010F000303122396D2AF1284
:020117000F4D8A
:070119001213821205071208
:06012000099F12143012C9
:06012600205A1221FD1217
:0A012C0022C81223C643870180E3B6
:0826480001020408102040808B
:0E013600C0E0C0D075D018758C70758A00E5D9
:050144002660021526F3
:06014900E5276002152706
:06014F00E52860021528FE
:06015500E52960021529F6
:06015B00E52A6002152AEE
:06016100E52B6002152BE6
:05016700D0D0D0E03211
:0E016C00758921758F00758C70758A00758DF0
:06017A0047D28CD2A9223D
:0E018000C0E0C0F0C082C083C0D075D008C2FD
:0C018E009853BAF1D201E599FA30E70865
:08019A008A821206FB0202AA90
:0501A200E4BA1B01049A
:0601A700FB6003753E0041
:0901AD00E53E24FB50030202AA06
:0501B600E53E253E2599
:0501BB003E9001C0733D
:0701C0000201CF0201DA0287
:0601C70002010202010228
:0201CD00026CC2
:0601CF00EB70030202AA1E
:0501D500053E0202AA34
:0501DA00BA5102800A89
:0501DF00BA5202800F7E
:0501E400BA5611800570
:0501E900753E02800DCF
:0501EE00753E038008CE
:0501F300753E048003CD
:0301F800753E0051
:0601FB00753F000202AA9C
:08020100E53F2440F8A60A05C0
:080209003F74FC253F40030295
:0202110002AA3F
:0C021300740F5540FB7C00C454F0FC7BD1
:0C021F0000740F5541FD8D0EE4FD420BF4
:0C022B00EE420C740F5542FDE4FEC4547A
:0E023700F0CDC4CD6DCD54F0CD6DFEED420B7B
:0C024500EE420C740F5543FD7E004BF59B
:060251002CEE4CF52DE53A
:060257003EB40302D20CCC
:05025D00D204D203757C
:060262002B00753C007545
:040268003E00803E96
:08026C00E53F2440F8A60A0555
:0A0274003F74FC253F502F740F5516
:06027E0040F53C747055D0
:0802840042FA740F55434AF5DC
:07028C003D900042740F5584
:0A02930041F0E54230E3047A0180F7
:01029D00025E
:02029E007A00E4
:0802A000EA24FF9207D2087561
:0202A8003E0016
:0B02AA00D0D0D083D082D0F0D0E03262
:0C02B500C0E0C0F0C0D075D010C299E5C8
:0602C1003AB53B02801576
:0602C700AA3B053BEA24FE
:0A02CD002EF8869975F00CE53B84CD
:0502D70085F03B8002F0
:0202DC00C20658
:0702DE00D0D0D0F0D0E032D7
:0802E500AA82AB3A053AEB24B2
:0A02ED002EF8A60275F00CE53A8425
:0402F70085F03A2232
:0702FB00200604D206D2998F
:0103020022D8
:0E03030075BD0075BF0B75BEF075BD03759816
:0C0311004075BAA0D29CD2ACD2EED20350
:09031D00752BC8D20975821B1270
:0503260002E50202FBEC
:0C032B00AA82900040E0FBA3E0FC756695
:0C03370014E4F5678B828C83C002C003C5
:0E034300C004122493AD82AE83D004D003D048
:0A03510002756614E4F5678B828CD8
:0E035B0083C002C0051225C1AB82AC83D00561
:0B036900D002EB75F005A4FBBD6400A2
:0E037400B3E433FC600A75F064ED842430FCC1
:020382008002F7
:020384007C20DB
:0E038600900043ECF075F064ED84ADF075F07E
:0E0394000AED842430FC900044F075F00AED70
:0E03A20084E5F02430FC900045F09000467495
:0E03B0002EF075F00AEB842430FC900047F02C
:0E03BE0075F00AEB84E5F02430FB900048F067
:0603CC008A6675670690C9
:0503D200004302129E31
:0703D700B205E4A20533F5B5
:0703DE00667582140210E4B1
:0E03E500AA82AB838A04EBCC25E0CC33FDEC7E
:0C03F30024F7FAED34FFFB756603E4F517
:0C03FF00678A828B83C002C0031225A411
:0C040B00AC82AD83D003D00275660DE416
:0C041700F5678A828B83C002C003C0041A
:0E042300C0051225A4AE82AF83D005D004D050
:0E04310003D0028A00EBC313C813C8C313C85C
:0E043F0013C8F9E82EFEE93FFF8F067F00EE9E
:0D044D002CFAEF3DFB75821BC002C00312AC
:0E045A0002E5D003D002758251C002C0031229
:0E04680002E5D003D002EBC4540FFC7D0074FB
:0E047600302CF582C002C0031202E5D003D084
:0E048400028B04740F5C2430F582C002C003AA
:0E0492001202E5D003D0028A04EBC4CCC4549D
:0E04A0000F6CCC540FCC6CCCFD53040F7D00C0
:0E04AE0074302CF582C002C0031202E5D003A8
:0D04BC00D00253020F7B0074302AF582122B
:0904C90002E575820D1202E50244
:0204D20002FB2B
:0C04D400900040E0FAA3E0FB300D0B307C
:0604E00005047C148002FB
:0204E6007C0197
:0204E800800B87
:0704EA003005047DEC8002E7
:0204F1007DFF8D
:0204F3008D0476
:0E04F500EC3395E0FDEC2AFAED3BFB8A828B9E
:04050300830203E587
:05050700100402806EEB
:0A050C00AA2CAB2DE4FCFDEBCCC4DF
:0E0516002354E0CCC423CC6CCC54E0CC6CFD60
:0E052400EAC42354E0FBEAC423541F4CFC7AC3
:080532000075668875671375FA
:0A053A0068007569008A828B838CCB
:0E054400F0ED12253FAA82AB83ACF0FD7432BD
:0C0552002AF582E43BF58375660AE4F5A7
:0A055E0067122493E5828583F09074
:0A0568000040F0A3E5F0F0D200120D
:050572000EE0C209C209
:0305770002D20BA2
:05057A00100B028018C7
:0A057F00E4A20A33F5667582221229
:0705890010E4E4A20233F5C7
:070590006675822F1210E4D2
:08059700300315E52B7011C2C1
:0B059F000375821B1202E575825212E8
:0505AA0002E51202FB56
:0605AF0010080302066AB9
:0B05B500C3E53C9402E433FAB40100FB
:0C05C000E433F5667582031210E4C3E515
:0905CC003C9403E433FAB401008D
:0C05D500E433F56675820A1210E4C3E5F9
:0905E1003C9404E433FAB4010077
:0C05EA00E433F5667582111210E4C3E5DD
:0905F6003C9407E433FAB401005F
:0C05FF00E433F5667582181210E4C3E5C1
:09060B003C940AE433FAB4010046
:0C061400E433F56675821F1210E4C3E5A4
:090620003C940DE433FAB401002E
:0B062900E433F5667582261210E43001
:0C0634000934900042E0FA602D75821B32
:0D0640001202E57582511202E575823F122B
:0C064D0002E575823F1202E575823F1243
:0C06590002E575823F1202E575820D1269
:0506650002E51202FB9A
:05066A00100C028013DA
:0E066F00900040E0FAA3E0FB900174EAF0A3D3
:05067D00EBF01221AEBC
:0E068200900174E0FAA3E0FB900040E0FCA3BE
:0E069000E0FDECB50208EDB503047401800135
:01069E00E477
:0C069F00FA758222C002121117D00292DC
:0706AB000EEA24FF920FA2EA
:0506B2000E300F01B342
:0B06B7005015758222121117920FA23D
:0A06C2000FB3E433F56675822202DF
:0206CC0010E438
:0106CE002209
:0306CF00D208222C
:0D06D20075821B1202E57582531202E502CB
:0206DF0002FB1C
:0C06E10075821B1202E53002047A4D8085
:0106ED00020A
:0206EE007A4E42
:0906F0008A821202E51202FBD21B
:0206F9000B22D2
:0406FB00AA8279074F
:0906FF00EA13FAE54D33F54DE56F
:050708004E33F54EE543
:05070D004F33F54FE53C
:050712005033F55030EA
:070717001108D54C0280031C
:03071E00020819B5
:08072100AC50AB4F530BC0E5D7
:070729004F30E503630CB73C
:0907300030E406630C5B630B80EE
:0907390030E306630C2D630BC0D4
:0907420030E206630CA1630BC058
:09074B0030E106630CE7630BC00A
:0907540030E006630CC4630BC025
:0B075D00E54E30E706630CD5630B404F
:0907680030E606630CDD630B8032
:0907710030E506630C6E630BC059
:09077A0030E406630C80630B40BF
:0607830030E303630CF7F4
:0907890030E206630C7B630B8077
:0907920030E106630C3D630BC06D
:09079B0030E006630CA9630BC0F9
:0B07A400E54D30E706630CE3630BC07B
:0907AF0030E606630CC6630BC0C2
:0C07B800BB00597E007851EC64F6601D17
:0A07C4000E7853EC64F560150E7812
:0C07CE0055EC6497600DEC64F360080EBD
:0707DA007857EC64967033C0
:0707E100A64F08A650EE65CB
:0607E80059702905595368
:0707EE005903BE031A8551F7
:0307F500448552E6
:0307F800458553E1
:0307FB00468554DC
:0307FE00478555D7
:03080100488556D1
:03080400498557CC
:030807004A8558C7
:03080A004BD210BE
:07080D00D211754C1A8005A1
:05081400C211E4F559DA
:04081900D90280037D
:03081D000206FFD1
:0108200022B5
:07082100AA82BA0102800562
:05082800BA042B80154D
:0A082D009000CE7401F09000CFE5BA
:0508370066F00567906A
:06083C0000D0E567F02288
:0A0842009000F17401F09000F2E55F
:05084C0066F005679055
:0508510000F3E567F073
:01085600227F
:05085700AA82BAE100D5
:05085C005003020988B1
:08086100EA2406500302098895
:0C086900900128E0FBE55AB50302800373
:0308750002097DF8
:04087800C2197B0125
:0A087C00C3EB955A501CEB2429F53C
:0C08860082E43401F583E0FC900129E0DD
:09089200FDECB50504D219800348
:03089B000B80DEF1
:07089E003019047B01800208
:0208A5007B00D6
:0908A7009000A3EBF020190302FC
:0208B00009330A
:0E08B200900129E0FB8B047D00746B2CFC741C
:0E08C000033DFDCC25E0CC33FD900040E0FE72
:0C08CE00A3E0FFECB5065AEDB50756207C
:0908DA00184F900099E4F07C0134
:0A08E300C3EC955A5042EC2429F5AD
:0C08ED0082E43401F583E0FD8D06BEFAC4
:0408F900030C802B41
:0308FD00BE010039
:0D0900004026EE24334021EEB50302801B9B
:0B090D00900099E0FF249AF582E4348A
:0C09180000F583EDF00F900099EFF0BFA8
:020924000900C8
:0209260050037C
:030928000C80B888
:04092B00D218804E10
:04092F00C218804A20
:07093300900099E4F07C0044
:0A093A00C3EC955A503DEC2429F55A
:0C09440082E43401F583E0FB8B06BEFA70
:04095000030C8026EE
:03095400BE0100E1
:0A0957004021EE2433401CBC0900CF
:0A096100501AEC249AF582E43400E9
:0E096B00F583EBF0900099E004FB900099EB0F
:01097900F08D
:03097A000C80BD31
:0B097D00EA2420900128F0755A0022A7
:0909880074E7255A4010AB5A0532
:080991005AEB2429F582E4343D
:0509990001F583EAF006
:01099E002236
:04099F001010012211
:0809A300900049E544F0A3E5D2
:0A09AB0045F0E54730E2047A0180D0
:0109B500023F
:0209B6007A00C5
:0809B800900094EAF0AA46E564
:0C09C00047C403CAC40354076ACA5407A2
:0E09CC00CA6ACAFB53021F7B00900097EAF034
:0C09DA00E547C423541FFA7B0053021FA2
:0A09E6007B00EAF55B6022E55BB4DC
:0409F0000102801B65
:0809F400E55BB40403020A9064
:0809FC00E55BB40603020B7574
:080A0400E55BB40803020C17C6
:030A0C00020C7465
:090A0F00E54630E4047B0180029D
:020A18007B0061
:090A1A00900098EBF075824A127D
:0C0A230022C074035546FB7C0025E0FC5B
:0A0A2F002420F582E43401F583E58C
:070A39004AF0A3E54BF09029
:0A0A4000011FE0FCEBB50402800783
:070A4A0090011FE4F080267B
:0E0A510090011F74012CF090011FE0FC24FCAA
:090A5F00501690011FE4F07566C9
:030A68002075678F
:050A6B00017568089010
:060A7000004B12229DD292
:010A7600126D
:070A7700E55B6003020C7453
:070A7E00854982120857AC04
:090A8500487D008C821208570222
:020A8E000C74E6
:0C0A90009000937401F0740F5546FC7D3B
:080A9C00008C03EB7002D2167E
:0A0AA400301527E546C45401FCE4B8
:090AAE00A21433FDB50402801707
:060AB700D21675662075E1
:060ABD0067409000531297
:080AC30022B39000CEE4F09094
:030ACB0000F1F047
:070ACE00E546A2E49214D2F8
:050AD5001520160302CC
:020ADA000C749A
:0B0ADC00EB2B25E0FC2453F582E434F2
:0A0AE70000F583E549FDF074012CD1
:0A0AF1002453F582E43400F583ADD0
:0A0AFB00487E00EDF074022C245335
:0A0B0500F582E43400F583E54BFDB2
:0A0B0F00F074032C2453F582E43443
:0A0B190000F583AC4A7D00ECF0907B
:0E0B230000CEE06021BB0F1E9000CFE0FC244E
:050B310053F566E434F9
:040B360000F56790CF
:060B3A0000D0E0F5689018
:090B400000D112229DE4F0A3F0A3
:0E0B49009000F1E06021BB0F1E9000F2E0FC76
:060B57002453F566E434AE
:040B5D0000F56790A8
:060B610000F3E0F56890CE
:090B670000F412229DE4F0A3F059
:050B7000D213020C7419
:020B75007C0002
:0E0B770090011EE0FDC3EC9D501EEC2CFE24F0
:0A0B850014F582E43401F583E0FE6C
:0A0B8F00A3E0FFEEB54A06EFB54BF8
:030B9900028003D4
:030B9C000C80D8F2
:070B9F00ECB50520BD0500C7
:0E0BA600501B74012DFC90011EF0ED2DFD245E
:090BB40014F582E43401F583E537
:060BBD004AF0A3E54BF035
:0A0BC300E54AB4A117E54BB44A124D
:0C0BCD009000A47401F0741F5546FC7DDC
:060BD900009000A5ECF005
:0A0BDF00E54AB4D721E54BB44B1CE6
:0C0BE9009000C57401F0741F5546FC7D9F
:0A0BF500009000C6ECF09000C7E588
:060BFF0048F0A3E549F0F7
:0A0C0500E54AB4466AE54BB4CD653C
:080C0F009000957401F0805D76
:0C0C17009000967401F0741F554AFC7D9B
:0C0C2300008C03E54BC4540FFC7D005313
:0C0C2F00040F7D0074015548FE7F00C4D6
:0C0C3B0054F0FE7F004204EF4205AD4A79
:0C0C4700E54BA2E7CD33CD33A2E7CD335F
:0C0C5300CD33CD5403FE53053F7E00E579
:0A0C5F004A30E506C3E49BFE800264
:020C69008B06F8
:070C6B008D668E678C82127A
:020C720023A0BD
:090C74009000A4E07003020D8958
:0C0C7D009000A5E0FCE55BB504028003DC
:030C8900020D89D0
:080C8C00AC469000A6ECF090CC
:070C940000A7E548F0A3E50D
:060C9B0049F09000A9E5FC
:090CA1004AF0A3E54BF0741F5565
:0C0CAA0046FC7D008C03EB0303543FFC70
:070CB600600DBC0102801A71
:050CBD00BC0302807C75
:030CC200020D8997
:080CC500AC4874035549FD9091
:0A0CCD0000ABECF0A3EDF0020D897E
:0A0CD7009000BAE0FC9000B9F09024
:090CE10000BBE0FC9000BAF0E554
:0C0CEA004BC423541FFC7D009000BBECA9
:0E0CF600F09000BEE0FCA3E0FD9000BCECF02E
:0E0D0400A3EDF09000C0E0FCA3E0FD9000BE67
:0C0D1200ECF0A3EDF09000C0E548F0A369
:090D1E00E549F09000C3E0FC90EF
:090D270000C2F09000C4E0FC9051
:080D300000C3F0AC4A7D009005
:060D380000C4ECF0804B4A
:0B0D3E0074035BFC6008BC0102800332
:030D4900BC023DAC
:0C0D4C00530303EB2B25E0FB24ADF582E4
:080D5800E43400F583AB48AC64
:0C0D6000497D008C068B057C007B00AFF9
:0A0D6C004AA84BE4F9FAEF4203E84D
:0E0D76004204E94205EA4206EBF0A3ECF0A3CA
:050D8400EDF0A3EEF00C
:090D89009000C5E07003020EA207
:0C0D92009000C6E0FAE55BB502028003A9
:030D9E00020EA2A0
:080DA100AA469000C9EAF09097
:070DA90000CAE548F0A3E5D4
:060DB00049F09000CCE5C3
:070DB6004AF0A3E54BF090A9
:0E0DBD0000CEE4F09000F1F0EAC45401FAE434
:090DCB00A21733FBB502028024DB
:060DD400B21775662075E0
:060DDA0067209000D11219
:080DE00022B39000D0E4F0758D
:060DE800662075672090F3
:060DEE0000F41222B39094
:040DF40000F3E4F034
:0C0DF800E546FAC40354F8FA530238E54B
:0C0E040049C4035407FB7C00530307E4BF
:0B0E1000FCFDEA4203ED4204AA48E5A5
:0C0E1B0049A2E7CA33CA33CA5401FC5391
:0A0E2700023FAC48E549C313CC13A9
:0A0E3100CCFD53043F7D008A668C5F
:070E3B00678B82120821E51C
:0B0E420048FAC42354E0FA530220E5F4
:0C0E4D004BC423541FFC7D0053041FE421
:0C0E5900FDFEEA4204EE42058C03AA4AAA
:0C0E6500E54BC403CAC40354076ACA5416
:0C0E710007CA6ACAFC53023F7C008A6674
:0A0E7D00741F554AFA7C008A678B47
:0C0E8700821208219000C9E0FAB40100BA
:0E0E9300E433FA30E3099000D1E4F09000F46B
:010EA100F060
:0A0EA200900097E0FAE4BA010104A1
:090EAC00F5667582061210E4904F
:0C0EB5000094E0FA900098E0FBB401000B
:0C0EC100E433FB5AF56675823F1210E422
:0C0ECD00900094E0FA900098E0FB5AF5C9
:070ED900667582530210E46C
:070EE0007566007567D690EE
:060EE70000491222B37560
:060EED0066207567089005
:060EF300004B1222B37552
:060EF900662075670890F9
:060EFF0001201222B3D213
:070F05001290011FE4F075DA
:060F0C00662075674090AD
:060F120000531222B3D2CD
:040F180013C215C229
:080F1C001675660075820612CD
:090F240010E475660075823F12AD
:090F2D0010E475660075825302A0
:020F360010E4C5
:0E0F3800900097E0541F25E0FA90265093CACF
:070F4600A3938A82F58322C8
:022650009026D2
:022652009926C7
:02265400A526B9
:02265600B326A9
:02265800C42696
:02265A00CA268E
:02265C00D22684
:02265E00E12673
:02266000F22660
:02266200FF2651
:022664000C2741
:02266600162735
:02266800302719
:02266A00402707
:02266C004F27F6
:02266E005F27E4
:022670006627DB
:022672007127CE
:022674008027BD
:022676008927B2
:022678009227A7
:02267A009F2798
:02267C00B02785
:02267E00B9277A
:02268000BE2773
:02268200CC2763
:02268400D82755
:02268600E52746
:02268800EE273B
:02268A00F62731
:04268C000128000021
:092690004B65696E20505459009D
:0C2699004E6163687269636874656E00CE
:0E26A500416B7475656C6C6520496E666F0044
:0E26B300536572766963652050726F677261BD
:0326C1006D6D003C
:0626C40053706F727400F8
:0826CA0042696C64756E670043
:0E26D200489772737069656C202B204C6974F8
:0126E00000F9
:0E26E1004B756C7475722B476573656C6C736A
:0326EF006368001D
:0D26F20057697373656E73636861667400E9
:0D26FF00556E74657268616C74756E6700CD
:0A270C00506F70204D7573696B006B
:0E271600526F636B204D7573696B556E746561
:0C2724007268616C74204D7573696B0065
:0E2730004C656963687465204B6C6173736956
:02273E006B002E
:0E27400045726E737465204B6C617373696B28
:01274E00008A
:0E274F005370657A69656C6C65204D75736911
:02275D006B000F
:07275F0057657474657200F8
:0B276600576972747363686166740049
:0E2771004B696E64657270726F6772616D6D98
:01277F000059
:09278000536F7A69616C65730006
:0927890052656C6967696F6E000E
:0D279200416E72756673656E64756E67004A
:0E279F005265697365696E666F726D6174696B
:0327AD006F6E004C
:0927B000467265697A65697400DE
:0527B9004A617A7A007C
:0E27BE00436F756E747279204D7573696B00F0
:0C27CC004C616E6465736D7573696B0081
:0D27D8004F6C64696573204D7573696B006B
:0927E500466F6C6B6C6F726500AD
:0827EE00466561747572650017
:0B27F600416C61726D2054657374002B
:0E280100416C61726D2120416C61726D21008D
:0E0F4D0075E29C43E240C2A4C294C2B07A3264
:060F5B00DAFED2947AC810
:0E0F6100DAFE758240120FE77582A1120FE7CB
:0E0F6F007582A2120FE77582C0120FE775821D
:0B0F7D002F120FE77582AF120FE71272
:060F88000FB6120FC3902A
:0C0F8E000149740FF090014A74ECF090DF
:090F9A00014B747FF012138C75F9
:020FA30029C85B
:050FA500E52970FC22AB
:0C0FAA007582AE120FE77582A5020FE7FA
:0D0FB60090016DE0FA74802AF582020FE7C9
:060FC30078007940742063
:0A0FC900F208D9FC90014E7908E40B
:070FD300F0A3D9FCD21A22A1
:060FDA00900142790CE4D5
:070FE000F0A3D9FCD21A2294
:050FE700C2B08582E3A9
:080FEC00E5E130E7FBF5E1222D
:050FF400D2B08582E38C
:080FF900E5E130E7FBF5E12220
:0E1001007582B8120FE7758211120FE7758223
:06100F0000120FE77A0059
:03101500BA0C0012
:0A10180050297B01EA2442FCE43475
:0210220001FDCE
:0E1024008C828D83E0FEEB5E60047E01800214
:021032007E003E
:0C1034008E82120FF4EB2BFB600280E4B4
:031040000A80D251
:01104300228A
:0A104400AA827B01E566248FFCE41C
:03104E00342CFD42
:0C105100EAC423541FFE2442F582E4345C
:0C105D0001F583E0FE74075A04F5F074FE
:0310690001800201
:02106C0025E07D
:0E106E00D5F0FBFFF4F852068C828D83E493DC
:08107C00F8EB586003EF420697
:0C108400EAC423541FFF2442F582E43428
:0C10900001F583EEF00AEB2BFBBB80B5F2
:01109C002231
:0C109D00AA8275F00AEA84F566758230BC
:0E10A900C002121044D00275F00AEA8485F0ED
:0B10B7006675823712104475F00AE5E0
:0810C2005C84F56675824112A1
:0A10CA00104475F00AE55C8485F01F
:0810D400667582481210447594
:0810DC00660175823E0210E47A
:0C10E400E582FAC423541F2442FBE434CC
:0C10F00001FC8B828C83E0FD74075A9099
:0C10FC00264893FAE5666005EA4205808C
:0111080005E1
:05110900EAF4FA5205B2
:09110E008B828C83EDF0D21A22D1
:0C111700E582FAC423541FFB2442F58239
:0C112300E43401F583E0FB5302078AF07E
:08112F0005F07A017C00800646
:06113700EA2AFAEC33FC89
:0E113D00D5F0F77D00EB5202ED5204E4BA004B
:05114B0004BC000104DA
:04115000FAB40100EC
:07115400E433F58224FF22C1
:02115B007A0018
:03115D00BA400095
:0311600040012229
:07116300EA540F6002801A3C
:0E116A00EAC4540FFB74B3C39BF582120FE767
:0C117800758211120FE7758200120FE75C
:0E1184008A82758300E0FB75F006A4FBACF0D8
:0A119200EAC423541F244EFDE43488
:0C119C0001FE74075A04F5F07401800293
:0211A80025E040
:0711AA00D5F0FBFF755D00AD
:0A11B10074FA255D402DA95D780059
:0C11BB00E92BF9E83CF8E9240FF582E884
:0C11C7003428F583E493F88D828E83E0D9
:0811D300F9EF5960036300FF0E
:0911DB008882120FF4055D80CD3D
:0411E4000A02115D8D
:0C11E800AA82AB83E567700474018001EB
:0111F400E416
:0711F50024FF921DC21CAC97
:0311FC0067AD6676
:0911FF00EC7006201D0302129B96
:0D1208008A828B83E493FE6029BEFF09D229
:081215001C0ABA00E50B80E29F
:0C121D00BEFE09C21C0ABA00D90B80D624
:0A1229008D827583000ABA00010BE4
:0712330053067FEEF0800B73
:0B123A00201D5E8D827583007420F083
:0C1245001CEDC423541FFE244EF582E46F
:0A1251003401F583E0FE301C147434
:09125B00075D04F5F07401800246
:0212640025E083
:08126600D5F0FBFF42068013E6
:0A126E0074075D04F5F074018002BE
:0212780025E06F
:07127A00D5F0FBF4FF520662
:0C128100EDC423541FFF244EF582E4341A
:09128D0001F583EEF00DBD4000F7
:0512960050030211FFEE
:03129B00D21A2242
:02129E00A86640
:0612A000E0B4D1027491DC
:0512A600B4D7027497AB
:0512AB00B4D9027499A2
:0712B000B400047420800368
:0312B700C2E7A3E8
:0A12BA00F208B840005003D567DCCD
:0312C400D21A2219
:0C12C700E566540F2430B43A00400224C5
:0112D3000713
:0612D400A882F2D21A22EA
:0A12DA00AA82E55EC4540FF5668A8F
:0E12E40082C0021212C7D00274012AF5828560
:0312F2005E660233
:0212F50012C71E
:0812F700AA8285605EC00212AC
:0B12FF0012DAD00274022AF582855F2B
:04130A005E0212DA93
:04130E00AA82AB61A3
:0C131200EB606CEB2A14FC75660AE4F535
:04131E0067F568F512
:0513220069856282856F
:0613270063838564F0E51C
:0C132D0065C002C003C0041224BCAD82E5
:0C133900AE83AFF0F8D004D003D0028DDA
:0C134500668C82C002C0031212C7D003E5
:09135100D00275660AE4F567F5A7
:04135A0068F5698544
:06135E00628285638385B5
:0913640064F0E565C002C003124B
:07136D00253F8582628583A4
:051374006385F064F543
:0813790065D003D0021B809136
:011381002249
:04138200101A01221A
:0613860012100102115BD0
:02138C007A00E5
:03138E00BA04009E
:0E139100504674B3C39AF582120FE7758211AD
:0E139F00120FE7758200120FE7EA75F060A4E6
:0513AD00FBACF07D0027
:0313B200BD60001B
:0E13B500501F8D067F00EE2BFEEF3CFFEE2456
:0A13C3000FF582EF342BF583E4935D
:0913CD00FEF582120FF40D80DC24
:0313D6000A80B5D5
:0A13D9007566017582031210E4022C
:0213E3001001F7
:0A13E5007566207567409000001245
:0613EF0022B37566FF75D4
:0613F500670890014E1292
:0613FB0022B37566FF75C8
:06140100670C900142128D
:0514070022B3D21A22FD
:0E280F00042A6AAA1E0004AA6A2A1E001C2AB5
:0E281D006AAA1A001CAA6A2A1A0000207E80ED
:0E282B00000000A07E0000001C2262A21C0023
:0E2839001CA262221C003C0242823E003C8235
:0E28470042023E00FE201008FE0078858587C4
:0E2855004800649292924C001F2A2A2A140016
:0E2863000020BE000000040282FC8000046A17
:0E287100AA6A1E0004AA2AAA1E001C6AAA6AED
:0E287F001A001CAA2AAA1A000040BE4000003F
:0E288D0000A03E8000001C62A2621C001CA283
:0E289B0022A21C003C4282423E003C8202828D
:0E28A9003E005E9050900E001825252724005A
:0E28B700122A2A2A24000010101010000020FF
:0E28C50040FE000000BC0101BE00000000004B
:0E28D30000000000FA00000000E00000E0003D
:0E28E10028FE28FE28002454FE5448006408F7
:0E28EF0010204C005CA2540814000020C00011
:0E28FD000000003844820000008244380000D1
:0E290B0054387C38540010107C10100000016D
:0E291900060000000010101010000000060064
:0E29270000000408102040007C8A92A27C0070
:0E293500002040FE000042868A92620044822A
:0E29430092926C00182848FE0800E4A2A2A29E
:0E2951009C003C5292928C0080809EA0C000A0
:0E295F006C9292926C0062929294780000004A
:0E296D00660000000001660000000010284413
:0E297B0082000024242424000082442810003E
:0E29890040809AA040007C82829A78007E9066
:0E29970090907E00FE9292926C007C82828272
:0E29A5004400FE8282827C00FE9292928200AA
:0E29B300FE90909080007C82828A4C00FE1084
:0E29C1001010FE000082FE820000040282FC64
:0E29CF008000FE1028448200FE020202020078
:0E29DD00FE403040FE00FE201008FE007C820E
:0E29EB0082827C00FE90909060007C8282844C
:0E29F9007A00FE9098946200649292924C00D4
:0E2A07008080FE808000FC020202FC00F804C9
:0E2A15000204F800FC020C02FC00C628102887
:0E2A2300C600C0201E20C000868A92A2C200FB
:0E2A310000FE82828200402010080400008215
:0E2A3F008282FE001010101010100101010123
:0E2A4D000101008040200000042A2A2A1E00F9
:0E2A5B00FE2222221C001C22222222001C220B
:0E2A69002222FE001C2A2A2A1A00107E9090BB
:0E2A77009000192525251E00FE2020201E009F
:0E2A85000020BE00000002010121BE0000FE84
:0E2A9300081422000080FE0000003E201E20DD
:0E2AA1001E003E2020201E001C2222221C00AF
:0E2AAF003F2424241800182424243F003E1045
:0E2ABD0020202000122A2A2A240020FC222297
:0E2ACB0022003C0202023E00380402043800E1
:0E2AD9003C020C023C002214081422003905B5
:0E2AE70005053E0022262A32220000106C82D5
:0E2AF50082000000FE0000000082826C1000D3
:0C2B0300808080808080000000000000C6
:0E2B0F000000000003060C091B1236246D495D
:0E2B1D0069494949692D2426331E0C091B32D3
:0E2B2B0026246D4949494969692D2436121B3B
:0E2B3900090C06030000000000000000010F60
:0E2B47003F3E38383838383838381800031B0D
:0E2B55003B3800000000010F3F3E3838383892
:0E2B6300383838381800031B3B380000000FCC
:0E2B71007BC38F3BE18F3F7FFFFFFFFEFCFC2D
:0E2B7F00F8FCFEFFF8C01F70C38F3F7FFFFF02
:0E2B8D00FFFEFCFCF8FCFFFFFFFF7F3F8FE127
:0E2B9B003B8FC37B0F0000070F7FFEF0E0E0D2
:0E2BA900E0E0E0E0C0C001073FFFFCC000001C
:0E2BB70000070F7FFEF0E0E0E0E0E0E0C0C0CD
:0E2BC50001073FFFFCC00000000000F0FEFF13
:0E2BD300FFFFFFFF9FC7F3D9CDE43612163483
:0E2BE10064CD19F3C70FFFFFFFFFFFFFFC6479
:0E2BEF003612163464CDD9F3C79FFFFFFFFFE7
:0E2BFD00FFFEF00007C4C485050406070707A5
:0E2C0B0007070604C4C6C7070707070404C569
:0E2C1900C48607070707070404070707C7C795
:0E2C2700C60405040607070000000080C0E098
:0E2C3500F0F8F8FCFCFCFEFEFEFEFEFEFEFECD
:0E2C4300FCFCFCF8F8F8F8FCFCFEFEFEFEFEC1
:0E2C5100FEFEFEFEFCFCFCF8F8F0E0C0800089
:0E2C5F000000FC0404BC9C0464FCFCFCFC04AF
:0E2C6D0004CCCC0404FCFCFCFC0404F4E40CD9
:0E2C7B001CFCFCFCFC0404FCFCFCFC1C0CE43B
:062C8900F4E40C1CFC0049
:0E2C8F006F28767C395D5F687F7D1010101015
:022C9D00101015
:09140C00E582900156F0D21E2287
:05141500101202800C22
:07141A007566087567089074
:05142100004B12129EB9
:04142600100001228F
:06142A0075820002032B95
:0A143000122023AA82E4BA4201044C
:0E143A00FB6014900156E0FC600DC28E53A2C0
:09144800DF900156E4F0D21E22EF
:0C145100BA4118B22790016FE0FC75F062
:0C145D0003A4902CE393FC900157F07561
:03146900286422D2
:08146C00E5287020752864904A
:0D1474000157E0FC6016EC14900157F09059
:0E1481000157E0FC700990016EE0FC6002C2B1
:01148F002735
:05149000101E02806047
:0D149500C002C003120FC3D003D0027C00C0
:0314A200BC11007A
:0D14A500504AEC2C25E0FD902C9F93FE900A
:0C14B2000156E0FFEEB50734ED249FFD6D
:0C14BE00E4342CFE8D828E83A3A3E49303
:0D14CA00FFA3E493F88D828E83A3E493F5D5
:0A14D700667567008F828883C002EB
:0D14E100C003C0041211E8D004D003D002F3
:0314EE000C80B1BE
:0414F100D212D20041
:0C14F500900156E0FC24D45003021FD8E4
:0D150100EC240983C0E0EC242F83C0E0221D
:02150E0066EA8B
:021510005D89F3
:0215120069442A
:02151400674C22
:021516004CD8AF
:02151800D8D821
:02151A00D8D81F
:02151C00D8D81D
:02151E00D8D81B
:02152000D8D819
:02152200D8D817
:02152400D8D815
:02152600D8D813
:02152800D8D811
:02152A00D8D80F
:02152C00BE926D
:02152E00866DC8
:02153000BE0BF0
:0215320075B290
:02153400758DB3
:02153600C932B8
:0215380076C17A
:02153A00151585
:02153C0016187F
:02153E00191B77
:021540001D1E6E
:021542001F1F69
:021544001F1F67
:021546001F1F65
:021548001F1F63
:02154A001F1F61
:02154C001F1F5F
:02154E001F1F5D
:021550001F1F5B
:021552001F1F59
:021554001F1F57
:021556001F1F55
:02155800151963
:02155A00161B5E
:02155C001C1F52
:02155E001E1855
:021560001F1F4B
:02156200191658
:02156400171D51
:0C156600C002C003121415D003D0021004
:0415720013028014CC
:0715760075661075673090E7
:0D157D000053C002C00312129ED003D00222
:05158A00BA21028013EC
:05158F00BA22028019E0
:05159400BA2302801AD9
:08159900EB700BBA430280174E
:0115A1002227
:0515A200C20D0204D49B
:0615A70075820102140C24
:0615AD001203D7D2032255
:0515B300D20D0204D47A
:0615B80075821E02140CF6
:0515BE00101302801073
:0715C300756600756740909A
:0915CA000053C00212129ED0026F
:0515D300BA22028006AF
:0515D800BA4302800788
:0115DD0022EB
:0615DE0075820302140CEB
:0615E40075820002140CE8
:0B15EA00C002121415D0023002067B74
:0515F500EF7C2C8004D6
:0415FA007BF37C2CD7
:0A15FE0075663D7567038B828C83D0
:0C160800C0021211E8D002BA2102800BCF
:05161400BA2202800E65
:05161900BA2302800F5E
:01161E0022A9
:08161F00D22975822902140C86
:0616270075820202140CA2
:05162D00B2020206E11B
:08163200900176E0FB8B62756C
:06163A00630075640075F9
:0A1640006500756101758221C0028A
:0A164A0012130ED002BA2202800132
:011654002273
:08165500C22975820002140C89
:0C165D00C002121415D002BA2102800B4A
:05166900BA2202800C12
:05166E00BA2302800D0B
:011673002254
:0616740075822002140C37
:06167A0075820302140C4E
:0616800075822A02140C21
:0E168600C002121415D002900049E0FBA3E050
:0C169400FC8C5E758213C0021212DAD0CA
:0C16A00002900049E0FBA3E0FC8B5E75AB
:0E16AC008215C0021212DAD002900097E0F50B
:0C16BA005E75821DC0021212DAD0029090
:0816C6000093E060067BF77C55
:0316CE002C800469
:0416D1007BF97C2CF9
:0A16D5007566237567008B828C8315
:0E16DF00C0021211E8D0029000C5E060067B48
:0516ED00F77C2C8004D5
:0416F2007BF97C2CD8
:0A16F6007566297567008B828C83EE
:0E170000C0021211E8D002900096E060067B55
:05170E00F77C2C8004B3
:041713007BF97C2CB6
:0A17170075662E7567008B828C83C7
:0E172100C0021211E8D002900095E060067B35
:05172F00F77C2C800492
:041734007BF97C2C95
:0A1738007566347567008B828C83A0
:0E174200C0021211E8D0029000A4E060067B05
:05175000F77C2C800471
:041755007BF97C2C74
:0A17590075663E7567008B828C8375
:0C176300C0021211E8D002BA220280017C
:01176F002257
:0617700075820202140C58
:0B177600C002121415D00275661F752A
:081781006701902CFBC002126D
:0A17890011E8D00290011EE0FB8B76
:051793006275630075A2
:0617980064007565007598
:0C179E00610175821FC00212130ED00200
:0217AA007B00C2
:0317AC00BB03007C
:0517AF00400302187D5B
:0E17B40074012BFCC454F0FC90011EE0FDC338
:0717C200EB9D4003021866D5
:0A17C900EB2BFD2414F582E434013B
:0A17D300F583E0FEA3E0FF8E628FB5
:0517DD00637564007556
:0A17E20065007561058C82C002C02D
:0E17EC0003C004C00512130ED005D004D003B4
:0C17FA00D00274062CFCED2414F582E4EF
:0C1806003401F583E0FDA3E0FEBDA10568
:05181200BE4A02801037
:08181700BDD705BE4B02801D88
:08181F00BD4657BECD54802ADE
:061827008C667567089055
:0E182D002CFDC002C0031211E8D003D00280CF
:01183B003D6F
:06183C008C667567089040
:0E1842002D04C002C0031211E8D003D00280B2
:01185000286F
:061851008C66756708902B
:0E1857002D0BC002C0031211E8D003D0028096
:01186500136F
:061866008C6675670E9010
:0D186C002D13C002C0031211E8D003D002FA
:041879000B0217AC9B
:05187D00BA2202800107
:011882002243
:0618830075820202140C44
:0C188900C002121415D002BA2102800B1C
:05189500BA2202800CE4
:05189A00BA2302800DDD
:01189F002226
:0618A00075821E02140C0B
:0618A60075820402140C1F
:0618AC0075822502140CF8
:0C18B200C002121415D0029000D0E0F526
:0518BE00677566109043
:0A18C3002CFBC0021211E8D00290C5
:0618CD0000D0E0F5677594
:0818D30066109000D1C0021262
:0E18DB00129ED0029000D0E0FB2411FC740F8E
:0518E9005CFDBD0A00DA
:0C18EE00400AECC4540F04FDC454F0FC8C
:0A18FA0074102BFBECC39BF5678B09
:0919040066902D14C002C004120B
:0B190D0011E8D004D0029000F3E0F5D8
:04191800678C6690E2
:0E191C002CFBC002C0041211E8D004D00290CF
:06192A0000F3E0F5678CFC
:09193000669000F4C002C004122C
:0E193900129ED004D0029000F3E0FB2CFCBC08
:0219470040005E
:0A19490050127440C39CF5678C66D1
:0A195300902D17C0021211E8D00217
:05195D00BA2202800126
:011962002262
:0619630075820302140C62
:0C196900C002121415D002BA2102800B3B
:05197500BA2202800C03
:05197A00BA2302800DFC
:01197F002245
:0619800075821F02140C29
:0619860075820502140C3D
:06198C0075822802140C14
:0C199200C002121415D002900097E0F57E
:0C199E005E75821AC0021212DAD002C07C
:0A19AA0002120F38D0027566207596
:0C19B4006710C0021211E8D002BA220233
:0219C0008001A4
:0119C2002202
:0619C30075820402140C01
:0919C900C002121415D0027B00CB
:0319D200BB09004E
:0519D5004003021B3875
:0E19DA0075F003EB84E5F0FDC454F02410FD1D
:0E19E80075F003EB84FE75F006A42DFCBE0224
:0219F600011CD2
:0D19F800900099E0FDC3EB9D4003021B2110
:0A1A0500EB249AF582E43400F58327
:0E1A0F00E0FD7E00746B2DFD74033EFEC3ED02
:0C1A1D0094E8EE9403B3E433FF60067F0E
:051A290019782D800476
:041A2E007F1B782D75
:0A1A32008C667567018F828883C0FF
:0E1A3C0002C003C004C005C0061211E8D006A7
:0C1A4A00D005D004D003D0027566E8750A
:0C1A560067038D828E83C002C003C004B1
:0E1A62001225C1AD82AE83D004D003D0027431
:0A1A7000012CFF75660AE4F5678D8E
:0E1A7A00828E83C002C003C004C005C006C037
:0E1A880007122493A882A983D007D006D005A8
:0A1A9600D004D003D00288628963F7
:071AA0007564007565007517
:0C1AA70061028F82C002C003C004C005B1
:0E1AB300C00612130ED006D005D004D003D00A
:0A1AC1000274032CF56675670190AE
:0D1ACB002D1DC002C003C004C005C00612DE
:0E1AD80011E8D006D005D004D003D00274046B
:0A1AE6002CFF75660AE4F5678D8297
:0E1AF0008E83C002C003C0071225C1AD82AEB6
:0A1AFE0083D007D003D0028D628E62
:051B0800637564007527
:0A1B0D0065007561018F82C002C0FF
:0A1B17000312130ED003D002801356
:061B21008C667567089058
:0D1B27002D13C002C0031211E8D003D0023C
:041B34000B0219D2B5
:051B3800BA2202800149
:011B3D002285
:061B3E0075820402140C84
:0C1B4400C002121415D002BA2102800B5E
:051B5000BA2202800C26
:051B5500BA2302800D1F
:011B5A002268
:061B5B0075822102140C4A
:061B610075820602140C5F
:061B670075822202140C3D
:0B1B6D009000A5E0FBC313FB8B62752A
:061B7800630075640075B6
:0A1B7E006500756102758202C00265
:0E1B880012130ED0029000A5E0FB30E0067BA9
:051B96001F7D2D8004FD
:041B9B007B217D2D00
:0A1B9F007566047567008B828D8364
:091BA900C0021211E8D0027C0018
:031BB200BC030071
:051BB5004003021C5872
:0C1BBA0074012CFBC454F0FDEC24B9F5C0
:0A1BC60082E43400F583E0FE8E6235
:071BD00075630075640075E8
:0A1BD70065007561028D82C002C036
:0E1BE10003C004C00512130ED005D004D003BB
:0C1BEF00D00274032DFEEC2CFF24BCF58A
:0C1BFB0082E43400F583E0FFA3E0F88FE3
:041C07006288637517
:061C0B0064007565007520
:0C1C110061058E82C002C003C004C00543
:0E1C1D0012130ED005D004D003D00274092D8E
:0A1C2B00FDEC24C2F582E43400F55C
:091C350083E0FE8E627563007508
:061C3E00640075650075ED
:0C1C440061038D82C002C00312130ED099
:081C500003D0028B04021BB259
:0E1C58009000A6E0FB741F5BFC0303543FF5F5
:0C1C660066758206C002C0041212C7D0CE
:0C1C720004D00274035CF566758208C0A3
:0E1C7E0002C0041212C7D004D002EC030354BB
:0E1C8C003FFC70229000A9E0FBA3E0FC530493
:061C9A001F8B628C6375D4
:061CA0006400756500758B
:0C1CA600610475820CC00212130ED00203
:051CB200BA22028001CE
:011CB700220A
:061CB80075820502140C08
:091CBE009000A4E060067BF77CB5
:031CC7002C80046A
:041CCA007BF97C2CFA
:0A1CCE007566067567008B828C8333
:0E1CD800C0021211E8D0029000ABE0FBA3E0C6
:061CE600FC8B628C6375AB
:061CEC006400756500753F
:0C1CF200610475820CC00212130ED002B7
:091CFE009000ADE0F562A3E0F5F1
:081D070063A3E0F564A3E0F51D
:0A1D0F0065756109758213C00212A8
:091D1900130ED0029000B1E0F5B8
:081D220062A3E0F563A3E0F504
:061D2A0064A3E0F56575FD
:0C1D30006109758223C00212130ED0025C
:091D3C009000B5E0F562A3E0F5AA
:081D450063A3E0F564A3E0F5DF
:0A1D4D0065756109758233C002124A
:091D5700130ED002BA2202800131
:011D60002260
:061D610075820502140C5E
:0E1D6700C002121415D002900173E060067BDA
:051D7500237C2D800419
:041D7A007B297C2D18
:0A1D7E007566307567068B828C8352
:0C1D8800C0021211E8D002BA2102800B48
:051D9400BA2202801CD0
:051D9900BA2302801DC9
:011D9E002222
:0A1D9F00900173E060047B008002F5
:021DA9007B01BC
:081DAB00900173EBF0D22C0251
:021DB30021AE5F
:061DB50075820702140C08
:061DBB0075822B02140CDE
:081DC100900042E0FB8B62750B
:061DC90063007564007563
:0A1DCF006500756102758217C002FD
:0A1DD90012130ED002756102E4F54A
:041DE30062F563F54D
:091DE70064F565758227C0021243
:0C1DF000130ED002900042E0FBB4010092
:0A1DFC00E433FB60067B2D7C2D8094
:011E060028B3
:0B1E0700900042E0FDBD01067D337E2F
:031E12002D80160A
:0B1E1500900042E0FFBF03067F38781A
:031E20002D80040E
:041E23007F3D782D5A
:041E27008F05880695
:041E2B008D038E0491
:0A1E2F0075661A7567068B828C83B6
:0C1E3900C0021211E8D002BA220280019F
:011E4500227A
:061E460075820602140C77
:0C1E4C00C002121415D002BA2102800B53
:051E5800BA2202800C1B
:051E5D00BA2302800D14
:011E6200225D
:061E630075822402140C3C
:061E690075820802140C52
:061E6F0075822302140C31
:0E1E7500C002121415D00290016EE060067BD0
:051E8300417C2D8004EC
:041E88007B467C2DEC
:0A1E8C007566207567078B828C8352
:0E1E9600C0021211E8D00290016FE0FB75F05F
:0A1EA40003A424E3FBE4342CFC8BC0
:0C1EAE00828C83A3E493FBA3E493FC75F7
:0A1EBA00662D7567008B828C83C0D3
:0B1EC400021211E8D002BA2102800BCC
:051ECF00BA2202801898
:051ED400BA2302801C8E
:011ED90022E6
:0A1EDA0090016EE060047B008002BE
:021EE4007B0180
:061EE60090016EEBF022FA
:091EEC001221AE75820702140CEC
:0D1EF50090016FE004FB90016FF0BB040052
:031F020050012269
:061F050090016FE4F022E0
:0C1F0B00C002121415D002BA2102800B93
:051F1700BA2202801750
:051F1C00BA2302801B46
:011F2100229D
:0C1F220090016DE0FB1B90016DEBF012D4
:051F2E0021CE020FB6F8
:091F33001221AE75820702140CA4
:0B1F3C0090016DE004FB90016DF012BD
:051F470021CE020FB6DF
:0C1F4C00C002121415D002BA2102800B52
:051F5800BA2202800C1A
:051F5D00BA2302800D13
:011F6200225C
:061F630075822602140C39
:061F690075820102140C58
:061F6F0075822702140C2C
:0E1F7500C0021213E5D002BA225F120FDAD2B8
:081F83002C1206CF7582080242
:021F8B00140C34
:0A1F8D00D28E43A220BA2102800A7E
:051F9700BA22028019CE
:051F9C00BA233F802282
:0B1FA100900170E004FA900170F01253
:091FAC0021CE900170E0F59622AF
:0E1FB5001221AEC28E53A2DF75820802140CF8
:0C1FC300900170E0FA1A900170EAF01230
:091FCF0021CE900170E0F596228C
:061FD80075820002140CEA
:011FDE0022E0
:062C9F0001104E2D29106A
:042CA5007D2D02106F
:042CA900B02D20101A
:042CAD00E52D0310FE
:042CB100162E0410C7
:042CB5004B2E1F1073
:042CB900802E051054
:042CBD008A2E21003A
:042CC100BF2E220000
:042CC500D02E0610F7
:042CC900032F2B00AA
:042CCD00382F071085
:042CD1005D2F24103F
:042CD500922F2320F7
:042CD900C52F0810EB
:042CDD00E82F2710A5
:022CE1001D30A4
:042CE3000350300565
:032CE70054300A5C
:032CEA005830144B
:022CED005C3059
:042CEF0045494E0005
:042CF30041555300F4
:022CF7002A00B1
:022CF9005E007B
:022CFB00FF00D8
:072CFD00524153414E540007
:072D040052546578742B00A6
:082D0B005244532D544D4300C6
:012D130000BF
:032D1400FE5E0060
:022D1700FE00BC
:022D1900310087
:022D1B00200096
:022D1D002E0086
:022D1F00420070
:022D210041006F
:062D23004C4F4B414C0037
:042D290055544300BA
:062D2D003C56302E380078
:052D330056302E3800AF
:052D380056302E3900A9
:042D3D00283F290002
:052D41004155544F0054
:082D46004D414E55454C4C0077
:0E2D4E005374616E642D6279202F20537475CA
:0E2D5C006D6D5354414E4420FF4D656E99FE3F
:0E2D6A0020204D555445204259202020FF3195
:052D78003E3E32FE00AA
:0E2D7D004142534348414C54454E20494E209C
:0E2D8B0020202020202053454B554E44454E1D
:0E2D990020202020202020FF204142425255C1
:092DA700434820FE2020202000FA
:0E2DB00020436F6465732F4170706C696B6116
:0E2DBE00742E434F44452020FF4D656E99FE54
:0E2DCC002020204F44414C4953544520FF32F3
:0B2DDA003E3E33FE204C4953544500A0
:0E2DE50050493A2020202020205054593A20F6
:0E2DF300202052543A202052542B3A202043E4
:0E2E0100543A2020544D433A202020202044F3
:072E0F004750533A20200058
:0E2E1600202020526164696F7465787420205A
:0E2E24002020525458542020FF4D656E99FE18
:0E2E3200202052542B20444953502020FF33BF
:0B2E40003E3E34FE2020444953500069
:0E2E4B005054592F416C7465726E2E4672659C
:0E2E5900712E505459202020FF4D656E99FEB9
:0E2E6700202020204146444953502020FF34B3
:0B2E75003E3E35FE2020444953500033
:0A2E80005054592D436F64653A0069
:0E2E8A00446966666572656E7469616C204706
:0E2E98005053444750532020FF4D656E99FE65
:0E2EA600202044475053524F48202020FF3533
:0B2EB4003E3E36FE2020205245460026
:0E2EBF00473A20202020202F20205A3A2020A1
:032ECD00202000C2
:0E2ED000444750533A20202049443A20202005
:0E2EDE002020783A20202020202020202020B4
:0E2EEC0020202020793A2020202020202020A5
:092EFA002020202020207A3A005B
:0E2F03005568727A6569742F53572D537461A7
:0E2F11006E64554852202020FF4D656E99FEDB
:0E2F1F0020202053572D202020202020FF3678
:0B2F2D003E3E37FE205354414E44004E
:0E2F3800536F6674776172652D56657273690A
:0E2F46006F6E526164696F3A202020202020B7
:092F5400202020204C43443A00E7
:0E2F5D004C69636874202F204B6F6E74726194
:0E2F6B0073744C4344202020FF4D656E99FE88
:0E2F790020204B4F4E544C4943485420FF3704
:0B2F87003E3E38FE2020524153540013
:0E2F9200202042656C6575636874756E67205B
:0E2FA000202020202020202020202020202063
:0E2FAE00202020204D4F44555320FF204F4B34
:092FBC0020FE20205A4549540072
:0E2FC500446973706C61792D4B6F6E7472618C
:0E2FD3007374203C3C202020FF204F4B20FE3A
:072FE1002020203E3E2000ED
:0E2FE8002020536572766963656D656E9920D1
:0E2FF6002020444953502020FF4D656E99FE67
:0E300400204B414C4942544553542020FF3884
:0B3012003E3E31FE20204354524C0093
:0E301D004B616C696272696572756E67206145
:0E302B0075663939363320487A20616E2050A0
:0E303900696E3132203C3C202020FF204F4B9E
:0930470020FE2020203E3E200066
:0430500020337300B6
:0430540020357300B0
:0430580031307300A0
:04305C00323073009B
:0A1FDF00C0D075D018C2E9D21F75FA
:051FE9002602D0D032F9
:0C1FEE00759307758607759400D2E922F0
:0C1FFA00AA82900168E0FB2458F582E404
:0C2006003401F583EAF090016874012BAE
:09201200F0900168E0FABA100038
:07201B004005900168E4F0AC
:01202200229B
:0E2023007A00900169E0FB900168E0FCEBB5EB
:042031000402802203
:0A203500EB2458F582E43401F58332
:0E203F00E0FA90016974012BF0900169E0FB5A
:03204D00BB1000C5
:072050004005900169E4F076
:032057008A822258
:04205A00201F012220
:05205E00E526600122EF
:0A206300752602A280B39223A28129
:09206D00B39224A282B392253043
:0C207600203990016AE0FA6013EA14902F
:0E208200016AF090016AE0FA70067582411260
:022090001FFA35
:0620920020232DC2209066
:07209800016AE0FAB4010047
:09209F00E433FA60047A118002B6
:0220A8007A219B
:0720AA008A82121FFA801167
:0620B10030230ED2209046
:0B20B700016A7432F0758281121FFA7A
:0C20C20030213990016BE0FA6013EA1441
:0E20CE0090016BF090016BE0FA700675824293
:0320DC00121FFAD6
:0620DF0020242DC2219017
:0720E500016BE0FAB40100F9
:0920EC00E433FA60047A12800268
:0220F5007A224D
:0720F7008A82121FFA80111A
:0620FE0030240ED22190F7
:0B210400016B7432F0758282121FFA2A
:0C210F0030223990016CE0FA6013EA14F1
:0E211B0090016CF090016CE0FA700675824342
:03212900121FFA88
:06212C0020252DC22290C7
:07213200016CE0FAB40100AA
:09213900E433FA60047A13800219
:022142007A23FE
:072144008A82121FFA8011CC
:06214B0030250ED22290A7
:0B215100016C7432F0758283121FFADB
:07215C0020200D20210A20C4
:092163002207C21F5394FED2E9C9
:01216C002250
:06216D0075F1008582F30C
:09217300E5F130E7FB85F2822260
:09217C0075F1008566F28582F31D
:06218500E5F130E7FB224A
:06218B007A6D7B017C006F
:03219100BC090086
:0E21940050158C8212216DAD828A828B83EDF4
:0921A200F0A3AA82AB830C80E6D5
:0321AB000221CE40
:0621AE007A6D7B017C004C
:0321B400BC090063
:0C21B70050148A828B83E0F566A3AA8294
:0A21C300AB838C8212217C0C80E7B4
:0121CD0022EF
:0821CE0090016DE0FABA120065
:0821D600500690016D7412F037
:0E21DE0090016DE0FA24E0500690016D741F30
:0121EC00F002
:0E21ED00900170E0FA24C05006900170743F1B
:0121FB00F0F3
:0121FC0022C0
:0A21FD00E5277072752764C2E9C27D
:0D2207008075C00175A12075A301758E05BD
:0E221400E58E30E3FBAAC5758E00D280539490
:0C222200FED2E9756601758250C0021200
:07222E0010E4D002BA950094
:06223500E433FBB40100DC
:0C223B00E433F56675824FC0021210E417
:05224700D002BAAF0057
:06224C00E433FBB40100C5
:0C225200E433F566758251C0021210E4FE
:05225E00D002BABC0033
:06226300E433FAB40100AF
:0A226900E433F5667582521210E4AA
:0C2273003026111223C2C29643840112CF
:08227F000FAA43870375A208B2
:06228700A227202801B38C
:0A228D00400DB228302803D296223B
:0522970075C800C296AD
:01229C00221F
:08229D0005A2856682856783B6
:0C22A500E0A305A2F0A305A2D568F50592
:0222B100A22267
:0422B300E566A867CD
:0422B700B800012248
:0522BB00F0A31880F7FC
:0822C000A882E608C618F62208
:0C22C800900177E0FA24FB500302239001
:0722D400EA2A2A9022DB73C5
:0722DB000222EA022328029F
:0622E200233202234E022C
:0222E800238948
:0A22EA003029079001777401F022FB
:0522F400E52A60012253
:0722F900752A6430010A9010
:072300000176E4F0C201C206
:022307002B2287
:04230900302B012252
:0E230D00900176E02401F0900176E0FBBB0326
:01231B0000C1
:03231C005001224B
:09231F009001777402F0D229222A
:0A232800D22A90017774012AF022F6
:0C2332009001767404F0752A647582290D
:09233E0012140C900177E0FA90F2
:07234700017774012AF02266
:09234E00202908900177E4F0D287
:022357002B2237
:08235900E52A7038752A649032
:092361000176E014900176F09081
:0A236A000176E0FA7025302A131204
:0623740006D2752A6490F8
:0C237A000177E0FA90017774012AF0224C
:03238600D226223A
:07238900E52A7008D22622AC
:05239000900177E4F06C
:012395002225
:0A23960075D2E175D30075D1612204
:0923A000E58290017AF0D22D9043
:0623A9000179E566F090E9
:0C23AF00017BE567F053D1FE43D10190A3
:0723BB000178E4F0D22C22AE
:0423C20053D1FE22D3
:0423C600202D0122A3
:0E23CA00E5D130E76A53D17F900178E024011D
:0923D800F0900178E0FABA3C0033
:0E23E100403B900178E4F0900179E02401F097
:0823EF00900179E0FABA3C000C
:0E23F7004023900179E4F090017AE0FA7B0037
:0A2405008A828B83A3756618E4F544
:09240F006712260EAA82AB83902D
:04241800017AEAF06B
:02241C00D22CC0
:0A241E00900173E060047A01800968
:09242800900178E0FB74015BFAFD
:082431008A6675823E1210E478
:04243900102C012240
:0E243D0090017AE0FA8A03900173E0603E7C21
:0E244B000074182AFAE43CFC90017BE0FDC20C
:0C245900D575F002ED30E704B2D5F404B4
:062465008430D502F404EE
:0E246B00FDA2D595E0FEED2AF582EE3CF5834C
:07247900756618E4F5671217
:08248000260EAA82AC838A0338
:09248800900179E0F55C8B820201
:02249100109D9C
:052493007A10E4FBFCDF
:0E249800E58225E0F582E58333F583EB33FB27
:0A24A600EC33FCEB9566F5F0EC95C5
:0924B000674006FCABF043820119
:0324B900DADD2247
:0624BC00F9E566456745E5
:0824C20068456960777800C3EA
:0A24CA0008E56920E73BE56625E020
:0624D400F566E56733F533
:0524DA0067E56833F521
:0524DF0068E56933F51A
:0824E40069E5829566E5839528
:0724EC0067E5F09568E99532
:0824F3006950D4C3E56913F53B
:0524FB0069E56813F51E
:0525000068E56713F51A
:0525050067E56613F517
:01250A00666A
:0A250B00E5829566FCE5839567FD07
:0A251500E5F09568FEE995694007BE
:07251F00F98EF08D838C8220
:07252600C3E56913F569E547
:05252D006813F568E5EC
:052532006713F567E5E9
:072537006613F566D8CEE93A
:01253E00227A
:08253F00FB7A20E4FCFDFEFF25
:0E254700E5822582F582E58333F583E5F033E6
:0B255500F5F0EB33FB4017DAE98042A1
:0E256000E5822582F582E58333F583E5F033CD
:05256E00F5F0EB33FB6A
:0E257300EC33FCED33FDEE33FEEF33FFEC9561
:0625810066ED9567EE9582
:0825870068EF95694013EC9523
:08258F0066FCED9567FDEE9579
:0925970068FEEF9569FF43820123
:0225A000DABEA1
:0225A200EB222A
:06009D00E478FFF6D8FD37
:08007B007900E94400601B7AE2
:050083000090306078E0
:030088007C75A0E4
:0A008B0001E493F2A308B800020597
:08009500A0D9F4DAF275A0FF16
:0B25A400E5828566F0A4C582C0F085CA
:0A25AF0067F0A4D0F025F0C5838585
:0825B90066F0A42583F58322DE
:0825C100E566456760467A01FA
:0725C900E56625E0F566E57B
:0925D00067334012F567E58295BE
:0A25D90066E583956740030A80E67B
:0325E300C3E567E6
:0725E60013F567E56613F52C
:0125ED006687
:0A25EE00C3E5829566F5F0E58395DC
:0825F800674005F58385F082C0
:07260000C3E56713F567E570
:062607006613F566DAE13E
:01260D0022AA
:0800A3007800E84400600A79CE
:0300AB000075A03D
:0600AE0000E4F309D8FC98
:0800B400783CE84401600C797E
:0B00BC0002900040E4F0A3D8FCD9FA49
:03006E0075817F1A
:0A007100122644E58260030200CA73
:0E260E00C2D5E58330E70DD2D5E4C39582F541
:06261C0082E49583F583C2
:0A262200E56730E70BE4C39566F5A9
:05262C0066E49567F56E
:012631006741
:0E2632001225C130D50BE4C39582F582E495E4
:0326400083F5839C
:012643002274
:042644007582002279
:00000001FF
